:1000160022859033E5905407B40705759F25800324
:10002600759F2022851890746412036A7E017F00F2
:1000360090E011E012037A90E010E02FFF50010EDD
:1000460022E590540390023525E073AE18AF19AC43
:100056001AAD1BEF2DFDEE3CFCAA1CAB1DED2BFBD8
:10006600EC3AFA8A1E8B1F8042AE18AF19AC1AAD55
:100076001B120354AA1CAB1DEF2BFBEE3AFA8A1E89
:100086008B1F8027AC18AD19AE1AAF1B12023DAC00
:100096001CAD1D1203908E1E8F1F800FAC18AD195C
:0B00A600AE1AAF1B12023D8C1E8D1F16
:080235000151016F018A01A2D1
:1000B100AE1EAF1F22751A00751900E5186020AE3B
:1000C10019AF1AE51875F002A4FDACF01DBDFF01D2
:1000D1001CEF2DFDEE3CFC8C198D1A151880DCAE41
:1000E10019AF1A2275210175220A75231475241975
:1000F100AE27AF28E5222FFF50010EE52312037A28
:10010100E524C395238522F0A4FDACF0EF2DFDEE8F
:100111003CFCE5218C068D071203888E298F2A75F8
:100121002B04752CD2752FD47530317531B27532DF
:100131006E752101E521D394025024AE2FAF3074A6
:10014100022FFF50010E8E2F8F30AE31AF3274036C
:100151001203888E318F327821740126F650D575BD
:100161001802112A8E2B8F2C85271885281985298D
:100171001A852A1B852B1C852C1D11478E2D8F2E30
:10018100AC2BAD2C12023DAC29AD2AED2FFFEC3E7C
:10019100FE740312037AE524048523F0A4FBAAF07C
:1001A1000BBB00010AE5228F018E048A068B071220
:1001B100037A0FBF00010EEF29F9EE3CFC8C2F8969
:1001C1003085221811B68E318F32A200B34036E548
:1001D10022252325248525F0A4FDACF08C298D2A28
:1001E100AA2FAB30740A2BFB50010A8A068B071227
:1001F10003548E2F8F30D297C200751803112A8EA7
:100201002B8F2C802DE522252325248525F084FFA5
:100211007E008E298F2AAC2FAD30740A2DFD50013E
:100221000C8C2F8D30C297D200751804112A8E2B99
:040231008F2C01E528
:10038800CFC39FFF50011E22C3EF9DFFEE9CFE22AC
:10023D00BC000FBE0008ED8FF084FFADF022E4FE90
:10024D00FF22BE000DEF60FE54F0606F20E7030249
:10025D0002F3EAC0E0EBC0E078017A0075F001EE40
:10026D0020E710EF25E0FFEE33FE0AC5F023C5F0C1
:10027D0030E7F0EA5407F9096A7A007B006001085B
:10028D00C3EC9E40167004ED9F4010ED9FFDEC9E5B
:10029D00FCE5F0CA4ACA03F5F08005E5F003F5F078
:1002AD00C3EE13FEEF13FFD9D77908CACBCAD8D046
:1002BD00EAFEEBFFD0E0FBD0E0FA22EC8FF084FCFD
:1002CD00ED54F045F0C48FF084FEEDC454F045F0CC
:1002DD00C48FF084FDEEC4FE54F02DFFEE540F3CA0
:1002ED00FEADF07C0022790078008FF0EC7E0820C6
:1002FD00E70DC3CD33CD33C933C9C833C8DEF08460
:10030D0049F9E5F08FF0BE00E6FD7C00E9FFE8FE5F
:01031D0022BD
:0E037A00F88FF0A4FFE5F0CE88F0A42EFE224E
:10035400EF8DF0A4F9A8F0EF8CF0A428F8EE8DF05E
:10036400A428FEE9FF22600D782B02037400783084
:06037400D8FED5E0F822DE
:0300030002031ED7
:03001300020339AC
:03000000020006F5
:0900060075813575D0000200E59A
:10031E00C0E0C0F0C083C082C0D075D008120016F5
:10032E00D0D0D082D083D0F0D0E032C0E0C0F0C0C8
:10033E0083C082C0D075D010120017D0D0D082D01A
:06034E0083D0F0D0E03284
:00000001FF
